
D:\STM32\Program\1.11_Odchudzanie\um0427\FWLib\project\RIDE\STM3210E-EVAL\stm32f10x_can.o:     file format elf32-littlearm
D:\STM32\Program\1.11_Odchudzanie\um0427\FWLib\project\RIDE\STM3210E-EVAL\stm32f10x_can.o

Disassembly of section .text.CAN_Init:

00000000 <CAN_Init>:
CAN_Init():
D:\STM32\Program\1.11_Odchudzanie\um0427\FWLib\library\src/stm32f10x_can.c:125
   0:	4a36      	ldr	r2, [pc, #216]	(dc <CAN_Init+0xdc>)
   2:	2301      	movs	r3, #1
   4:	6013      	str	r3, [r2, #0]
D:\STM32\Program\1.11_Odchudzanie\um0427\FWLib\library\src/stm32f10x_can.c:128
   6:	6853      	ldr	r3, [r2, #4]
D:\STM32\Program\1.11_Odchudzanie\um0427\FWLib\library\src/stm32f10x_can.c:107
   8:	4601      	mov	r1, r0
D:\STM32\Program\1.11_Odchudzanie\um0427\FWLib\library\src/stm32f10x_can.c:128
   a:	f013 0001 	ands.w	r0, r3, #1	; 0x1
   e:	d063      	beq.n	d8 <CAN_Init+0xd8>
D:\STM32\Program\1.11_Odchudzanie\um0427\FWLib\library\src/stm32f10x_can.c:135
  10:	780b      	ldrb	r3, [r1, #0]
  12:	2b01      	cmp	r3, #1
D:\STM32\Program\1.11_Odchudzanie\um0427\FWLib\library\src/stm32f10x_can.c:137
  14:	bf0b      	itete	eq
  16:	6813      	ldreq	r3, [r2, #0]
D:\STM32\Program\1.11_Odchudzanie\um0427\FWLib\library\src/stm32f10x_can.c:141
  18:	6813      	ldrne	r3, [r2, #0]
D:\STM32\Program\1.11_Odchudzanie\um0427\FWLib\library\src/stm32f10x_can.c:137
  1a:	f043 0380 	orreq.w	r3, r3, #128	; 0x80
D:\STM32\Program\1.11_Odchudzanie\um0427\FWLib\library\src/stm32f10x_can.c:141
  1e:	f023 0380 	bicne.w	r3, r3, #128	; 0x80
  22:	6013      	str	r3, [r2, #0]
D:\STM32\Program\1.11_Odchudzanie\um0427\FWLib\library\src/stm32f10x_can.c:145
  24:	784b      	ldrb	r3, [r1, #1]
  26:	2b01      	cmp	r3, #1
  28:	d104      	bne.n	34 <CAN_Init+0x34>
D:\STM32\Program\1.11_Odchudzanie\um0427\FWLib\library\src/stm32f10x_can.c:147
  2a:	4a2c      	ldr	r2, [pc, #176]	(dc <CAN_Init+0xdc>)
  2c:	6813      	ldr	r3, [r2, #0]
  2e:	f043 0340 	orr.w	r3, r3, #64	; 0x40
  32:	e003      	b.n	3c <CAN_Init+0x3c>
D:\STM32\Program\1.11_Odchudzanie\um0427\FWLib\library\src/stm32f10x_can.c:151
  34:	4a29      	ldr	r2, [pc, #164]	(dc <CAN_Init+0xdc>)
  36:	6813      	ldr	r3, [r2, #0]
  38:	f023 0340 	bic.w	r3, r3, #64	; 0x40
  3c:	6013      	str	r3, [r2, #0]
D:\STM32\Program\1.11_Odchudzanie\um0427\FWLib\library\src/stm32f10x_can.c:155
  3e:	788b      	ldrb	r3, [r1, #2]
  40:	2b01      	cmp	r3, #1
  42:	d104      	bne.n	4e <CAN_Init+0x4e>
D:\STM32\Program\1.11_Odchudzanie\um0427\FWLib\library\src/stm32f10x_can.c:157
  44:	4a25      	ldr	r2, [pc, #148]	(dc <CAN_Init+0xdc>)
  46:	6813      	ldr	r3, [r2, #0]
  48:	f043 0320 	orr.w	r3, r3, #32	; 0x20
  4c:	e003      	b.n	56 <CAN_Init+0x56>
D:\STM32\Program\1.11_Odchudzanie\um0427\FWLib\library\src/stm32f10x_can.c:161
  4e:	4a23      	ldr	r2, [pc, #140]	(dc <CAN_Init+0xdc>)
  50:	6813      	ldr	r3, [r2, #0]
  52:	f023 0320 	bic.w	r3, r3, #32	; 0x20
  56:	6013      	str	r3, [r2, #0]
D:\STM32\Program\1.11_Odchudzanie\um0427\FWLib\library\src/stm32f10x_can.c:165
  58:	78cb      	ldrb	r3, [r1, #3]
  5a:	2b01      	cmp	r3, #1
  5c:	d104      	bne.n	68 <CAN_Init+0x68>
D:\STM32\Program\1.11_Odchudzanie\um0427\FWLib\library\src/stm32f10x_can.c:167
  5e:	4a1f      	ldr	r2, [pc, #124]	(dc <CAN_Init+0xdc>)
  60:	6813      	ldr	r3, [r2, #0]
  62:	f043 0310 	orr.w	r3, r3, #16	; 0x10
  66:	e003      	b.n	70 <CAN_Init+0x70>
D:\STM32\Program\1.11_Odchudzanie\um0427\FWLib\library\src/stm32f10x_can.c:171
  68:	4a1c      	ldr	r2, [pc, #112]	(dc <CAN_Init+0xdc>)
  6a:	6813      	ldr	r3, [r2, #0]
  6c:	f023 0310 	bic.w	r3, r3, #16	; 0x10
  70:	6013      	str	r3, [r2, #0]
D:\STM32\Program\1.11_Odchudzanie\um0427\FWLib\library\src/stm32f10x_can.c:175
  72:	790b      	ldrb	r3, [r1, #4]
  74:	2b01      	cmp	r3, #1
  76:	d104      	bne.n	82 <CAN_Init+0x82>
D:\STM32\Program\1.11_Odchudzanie\um0427\FWLib\library\src/stm32f10x_can.c:177
  78:	4a18      	ldr	r2, [pc, #96]	(dc <CAN_Init+0xdc>)
  7a:	6813      	ldr	r3, [r2, #0]
  7c:	f043 0308 	orr.w	r3, r3, #8	; 0x8
  80:	e003      	b.n	8a <CAN_Init+0x8a>
D:\STM32\Program\1.11_Odchudzanie\um0427\FWLib\library\src/stm32f10x_can.c:181
  82:	4a16      	ldr	r2, [pc, #88]	(dc <CAN_Init+0xdc>)
  84:	6813      	ldr	r3, [r2, #0]
  86:	f023 0308 	bic.w	r3, r3, #8	; 0x8
  8a:	6013      	str	r3, [r2, #0]
D:\STM32\Program\1.11_Odchudzanie\um0427\FWLib\library\src/stm32f10x_can.c:185
  8c:	794b      	ldrb	r3, [r1, #5]
  8e:	2b01      	cmp	r3, #1
  90:	d104      	bne.n	9c <CAN_Init+0x9c>
D:\STM32\Program\1.11_Odchudzanie\um0427\FWLib\library\src/stm32f10x_can.c:187
  92:	4a12      	ldr	r2, [pc, #72]	(dc <CAN_Init+0xdc>)
  94:	6813      	ldr	r3, [r2, #0]
  96:	f043 0304 	orr.w	r3, r3, #4	; 0x4
  9a:	e003      	b.n	a4 <CAN_Init+0xa4>
D:\STM32\Program\1.11_Odchudzanie\um0427\FWLib\library\src/stm32f10x_can.c:191
  9c:	4a0f      	ldr	r2, [pc, #60]	(dc <CAN_Init+0xdc>)
  9e:	6813      	ldr	r3, [r2, #0]
  a0:	f023 0304 	bic.w	r3, r3, #4	; 0x4
  a4:	6013      	str	r3, [r2, #0]
D:\STM32\Program\1.11_Odchudzanie\um0427\FWLib\library\src/stm32f10x_can.c:195
  a6:	798a      	ldrb	r2, [r1, #6]
  a8:	79cb      	ldrb	r3, [r1, #7]
  aa:	0792      	lsls	r2, r2, #30
  ac:	ea42 6203 	orr.w	r2, r2, r3, lsl #24
  b0:	7a0b      	ldrb	r3, [r1, #8]
  b2:	ea42 4203 	orr.w	r2, r2, r3, lsl #16
  b6:	7a4b      	ldrb	r3, [r1, #9]
  b8:	ea42 5203 	orr.w	r2, r2, r3, lsl #20
  bc:	894b      	ldrh	r3, [r1, #10]
  be:	4907      	ldr	r1, [pc, #28]	(dc <CAN_Init+0xdc>)
  c0:	3b01      	subs	r3, #1
  c2:	431a      	orrs	r2, r3
  c4:	61ca      	str	r2, [r1, #28]
D:\STM32\Program\1.11_Odchudzanie\um0427\FWLib\library\src/stm32f10x_can.c:202
  c6:	680b      	ldr	r3, [r1, #0]
  c8:	f023 0301 	bic.w	r3, r3, #1	; 0x1
  cc:	600b      	str	r3, [r1, #0]
D:\STM32\Program\1.11_Odchudzanie\um0427\FWLib\library\src/stm32f10x_can.c:210
  ce:	684b      	ldr	r3, [r1, #4]
  d0:	f003 0301 	and.w	r3, r3, #1	; 0x1
  d4:	f083 0001 	eor.w	r0, r3, #1	; 0x1
D:\STM32\Program\1.11_Odchudzanie\um0427\FWLib\library\src/stm32f10x_can.c:218
  d8:	4770      	bx	lr
  da:	46c0      	nop			(mov r8, r8)
  dc:	40006400 	.word	0x40006400
Disassembly of section .text.CAN_FilterInit:

00000000 <CAN_FilterInit>:
CAN_FilterInit():
D:\STM32\Program\1.11_Odchudzanie\um0427\FWLib\library\src/stm32f10x_can.c:244
   0:	493c      	ldr	r1, [pc, #240]	(f4 <CAN_FilterInit+0xf4>)
D:\STM32\Program\1.11_Odchudzanie\um0427\FWLib\library\src/stm32f10x_can.c:230
   2:	b510      	push	{r4, lr}
D:\STM32\Program\1.11_Odchudzanie\um0427\FWLib\library\src/stm32f10x_can.c:244
   4:	f8d1 3200 	ldr.w	r3, [r1, #512]
D:\STM32\Program\1.11_Odchudzanie\um0427\FWLib\library\src/stm32f10x_can.c:240
   8:	f890 e000 	ldrb.w	lr, [r0]
D:\STM32\Program\1.11_Odchudzanie\um0427\FWLib\library\src/stm32f10x_can.c:244
   c:	f043 0301 	orr.w	r3, r3, #1	; 0x1
  10:	f8c1 3200 	str.w	r3, [r1, #512]
D:\STM32\Program\1.11_Odchudzanie\um0427\FWLib\library\src/stm32f10x_can.c:247
  14:	2301      	movs	r3, #1
  16:	fa03 f30e 	lsl.w	r3, r3, lr
  1a:	f8d1 221c 	ldr.w	r2, [r1, #540]
  1e:	b29c      	uxth	r4, r3
  20:	ea6f 0c04 	mvn.w	ip, r4
  24:	ea0c 0202 	and.w	r2, ip, r2
  28:	f8c1 221c 	str.w	r2, [r1, #540]
D:\STM32\Program\1.11_Odchudzanie\um0427\FWLib\library\src/stm32f10x_can.c:250
  2c:	7883      	ldrb	r3, [r0, #2]
  2e:	b9a3      	cbnz	r3, 5a <CAN_FilterInit+0x5a>
D:\STM32\Program\1.11_Odchudzanie\um0427\FWLib\library\src/stm32f10x_can.c:253
  30:	f8d1 320c 	ldr.w	r3, [r1, #524]
D:\STM32\Program\1.11_Odchudzanie\um0427\FWLib\library\src/stm32f10x_can.c:257
  34:	8942      	ldrh	r2, [r0, #10]
D:\STM32\Program\1.11_Odchudzanie\um0427\FWLib\library\src/stm32f10x_can.c:253
  36:	ea0c 0303 	and.w	r3, ip, r3
  3a:	f8c1 320c 	str.w	r3, [r1, #524]
D:\STM32\Program\1.11_Odchudzanie\um0427\FWLib\library\src/stm32f10x_can.c:257
  3e:	88c3      	ldrh	r3, [r0, #6]
D:\STM32\Program\1.11_Odchudzanie\um0427\FWLib\library\src/stm32f10x_can.c:263
  40:	8901      	ldrh	r1, [r0, #8]
D:\STM32\Program\1.11_Odchudzanie\um0427\FWLib\library\src/stm32f10x_can.c:257
  42:	ea43 4302 	orr.w	r3, r3, r2, lsl #16
  46:	ea4f 02ce 	mov.w	r2, lr, lsl #3
  4a:	f102 4280 	add.w	r2, r2, #1073741824	; 0x40000000
  4e:	f502 42c8 	add.w	r2, r2, #25600	; 0x6400
  52:	f8c2 3240 	str.w	r3, [r2, #576]
D:\STM32\Program\1.11_Odchudzanie\um0427\FWLib\library\src/stm32f10x_can.c:263
  56:	8883      	ldrh	r3, [r0, #4]
  58:	e015      	b.n	86 <CAN_FilterInit+0x86>
D:\STM32\Program\1.11_Odchudzanie\um0427\FWLib\library\src/stm32f10x_can.c:267
  5a:	2b01      	cmp	r3, #1
  5c:	d117      	bne.n	8e <CAN_FilterInit+0x8e>
D:\STM32\Program\1.11_Odchudzanie\um0427\FWLib\library\src/stm32f10x_can.c:270
  5e:	f8d1 320c 	ldr.w	r3, [r1, #524]
D:\STM32\Program\1.11_Odchudzanie\um0427\FWLib\library\src/stm32f10x_can.c:273
  62:	8882      	ldrh	r2, [r0, #4]
D:\STM32\Program\1.11_Odchudzanie\um0427\FWLib\library\src/stm32f10x_can.c:270
  64:	ea44 0303 	orr.w	r3, r4, r3
  68:	f8c1 320c 	str.w	r3, [r1, #524]
D:\STM32\Program\1.11_Odchudzanie\um0427\FWLib\library\src/stm32f10x_can.c:273
  6c:	88c3      	ldrh	r3, [r0, #6]
D:\STM32\Program\1.11_Odchudzanie\um0427\FWLib\library\src/stm32f10x_can.c:278
  6e:	8901      	ldrh	r1, [r0, #8]
D:\STM32\Program\1.11_Odchudzanie\um0427\FWLib\library\src/stm32f10x_can.c:273
  70:	ea43 4302 	orr.w	r3, r3, r2, lsl #16
  74:	ea4f 02ce 	mov.w	r2, lr, lsl #3
  78:	f102 4280 	add.w	r2, r2, #1073741824	; 0x40000000
  7c:	f502 42c8 	add.w	r2, r2, #25600	; 0x6400
  80:	f8c2 3240 	str.w	r3, [r2, #576]
D:\STM32\Program\1.11_Odchudzanie\um0427\FWLib\library\src/stm32f10x_can.c:278
  84:	8943      	ldrh	r3, [r0, #10]
  86:	ea43 4301 	orr.w	r3, r3, r1, lsl #16
  8a:	f8c2 3244 	str.w	r3, [r2, #580]
D:\STM32\Program\1.11_Odchudzanie\um0427\FWLib\library\src/stm32f10x_can.c:285
  8e:	7843      	ldrb	r3, [r0, #1]
  90:	b92b      	cbnz	r3, 9e <CAN_FilterInit+0x9e>
D:\STM32\Program\1.11_Odchudzanie\um0427\FWLib\library\src/stm32f10x_can.c:288
  92:	4a18      	ldr	r2, [pc, #96]	(f4 <CAN_FilterInit+0xf4>)
  94:	f8d2 3204 	ldr.w	r3, [r2, #516]
  98:	ea0c 0303 	and.w	r3, ip, r3
  9c:	e004      	b.n	a8 <CAN_FilterInit+0xa8>
D:\STM32\Program\1.11_Odchudzanie\um0427\FWLib\library\src/stm32f10x_can.c:293
  9e:	4a15      	ldr	r2, [pc, #84]	(f4 <CAN_FilterInit+0xf4>)
  a0:	f8d2 3204 	ldr.w	r3, [r2, #516]
  a4:	ea44 0303 	orr.w	r3, r4, r3
  a8:	f8c2 3204 	str.w	r3, [r2, #516]
D:\STM32\Program\1.11_Odchudzanie\um0427\FWLib\library\src/stm32f10x_can.c:297
  ac:	8983      	ldrh	r3, [r0, #12]
  ae:	b92b      	cbnz	r3, bc <CAN_FilterInit+0xbc>
D:\STM32\Program\1.11_Odchudzanie\um0427\FWLib\library\src/stm32f10x_can.c:300
  b0:	4a10      	ldr	r2, [pc, #64]	(f4 <CAN_FilterInit+0xf4>)
  b2:	f8d2 3214 	ldr.w	r3, [r2, #532]
  b6:	ea0c 0303 	and.w	r3, ip, r3
  ba:	e006      	b.n	ca <CAN_FilterInit+0xca>
D:\STM32\Program\1.11_Odchudzanie\um0427\FWLib\library\src/stm32f10x_can.c:302
  bc:	2b01      	cmp	r3, #1
  be:	d106      	bne.n	ce <CAN_FilterInit+0xce>
D:\STM32\Program\1.11_Odchudzanie\um0427\FWLib\library\src/stm32f10x_can.c:305
  c0:	4a0c      	ldr	r2, [pc, #48]	(f4 <CAN_FilterInit+0xf4>)
  c2:	f8d2 3214 	ldr.w	r3, [r2, #532]
  c6:	ea44 0303 	orr.w	r3, r4, r3
  ca:	f8c2 3214 	str.w	r3, [r2, #532]
D:\STM32\Program\1.11_Odchudzanie\um0427\FWLib\library\src/stm32f10x_can.c:309
  ce:	7b83      	ldrb	r3, [r0, #14]
  d0:	2b01      	cmp	r3, #1
  d2:	d106      	bne.n	e2 <CAN_FilterInit+0xe2>
D:\STM32\Program\1.11_Odchudzanie\um0427\FWLib\library\src/stm32f10x_can.c:311
  d4:	4a07      	ldr	r2, [pc, #28]	(f4 <CAN_FilterInit+0xf4>)
  d6:	f8d2 321c 	ldr.w	r3, [r2, #540]
  da:	ea44 0303 	orr.w	r3, r4, r3
  de:	f8c2 321c 	str.w	r3, [r2, #540]
D:\STM32\Program\1.11_Odchudzanie\um0427\FWLib\library\src/stm32f10x_can.c:315
  e2:	4a04      	ldr	r2, [pc, #16]	(f4 <CAN_FilterInit+0xf4>)
  e4:	f8d2 3200 	ldr.w	r3, [r2, #512]
  e8:	f023 0301 	bic.w	r3, r3, #1	; 0x1
  ec:	f8c2 3200 	str.w	r3, [r2, #512]
D:\STM32\Program\1.11_Odchudzanie\um0427\FWLib\library\src/stm32f10x_can.c:316
  f0:	bd10      	pop	{r4, pc}
  f2:	46c0      	nop			(mov r8, r8)
  f4:	40006400 	.word	0x40006400
Disassembly of section .text.CAN_StructInit:

00000000 <CAN_StructInit>:
CAN_StructInit():
D:\STM32\Program\1.11_Odchudzanie\um0427\FWLib\library\src/stm32f10x_can.c:331
   0:	2300      	movs	r3, #0
   2:	7003      	strb	r3, [r0, #0]
D:\STM32\Program\1.11_Odchudzanie\um0427\FWLib\library\src/stm32f10x_can.c:334
   4:	7043      	strb	r3, [r0, #1]
D:\STM32\Program\1.11_Odchudzanie\um0427\FWLib\library\src/stm32f10x_can.c:337
   6:	7083      	strb	r3, [r0, #2]
D:\STM32\Program\1.11_Odchudzanie\um0427\FWLib\library\src/stm32f10x_can.c:340
   8:	70c3      	strb	r3, [r0, #3]
D:\STM32\Program\1.11_Odchudzanie\um0427\FWLib\library\src/stm32f10x_can.c:343
   a:	7103      	strb	r3, [r0, #4]
D:\STM32\Program\1.11_Odchudzanie\um0427\FWLib\library\src/stm32f10x_can.c:346
   c:	7143      	strb	r3, [r0, #5]
D:\STM32\Program\1.11_Odchudzanie\um0427\FWLib\library\src/stm32f10x_can.c:349
   e:	7183      	strb	r3, [r0, #6]
D:\STM32\Program\1.11_Odchudzanie\um0427\FWLib\library\src/stm32f10x_can.c:352
  10:	71c3      	strb	r3, [r0, #7]
D:\STM32\Program\1.11_Odchudzanie\um0427\FWLib\library\src/stm32f10x_can.c:355
  12:	3303      	adds	r3, #3
  14:	7203      	strb	r3, [r0, #8]
D:\STM32\Program\1.11_Odchudzanie\um0427\FWLib\library\src/stm32f10x_can.c:358
  16:	3b01      	subs	r3, #1
  18:	7243      	strb	r3, [r0, #9]
D:\STM32\Program\1.11_Odchudzanie\um0427\FWLib\library\src/stm32f10x_can.c:361
  1a:	f04f 0301 	mov.w	r3, #1	; 0x1
  1e:	8143      	strh	r3, [r0, #10]
D:\STM32\Program\1.11_Odchudzanie\um0427\FWLib\library\src/stm32f10x_can.c:362
  20:	4770      	bx	lr
  22:	46c0      	nop			(mov r8, r8)
Disassembly of section .text.CAN_ITConfig:

00000000 <CAN_ITConfig>:
CAN_ITConfig():
D:\STM32\Program\1.11_Odchudzanie\um0427\FWLib\library\src/stm32f10x_can.c:385
   0:	b121      	cbz	r1, c <CAN_ITConfig+0xc>
D:\STM32\Program\1.11_Odchudzanie\um0427\FWLib\library\src/stm32f10x_can.c:388
   2:	4a05      	ldr	r2, [pc, #20]	(18 <CAN_ITConfig+0x18>)
   4:	6953      	ldr	r3, [r2, #20]
   6:	ea40 0303 	orr.w	r3, r0, r3
   a:	e003      	b.n	14 <CAN_ITConfig+0x14>
D:\STM32\Program\1.11_Odchudzanie\um0427\FWLib\library\src/stm32f10x_can.c:393
   c:	4a02      	ldr	r2, [pc, #8]	(18 <CAN_ITConfig+0x18>)
   e:	6953      	ldr	r3, [r2, #20]
  10:	ea23 0300 	bic.w	r3, r3, r0
  14:	6153      	str	r3, [r2, #20]
D:\STM32\Program\1.11_Odchudzanie\um0427\FWLib\library\src/stm32f10x_can.c:395
  16:	4770      	bx	lr
  18:	40006400 	.word	0x40006400
Disassembly of section .text.CAN_Transmit:

00000000 <CAN_Transmit>:
CAN_Transmit():
D:\STM32\Program\1.11_Odchudzanie\um0427\FWLib\library\src/stm32f10x_can.c:418
   0:	4a3a      	ldr	r2, [pc, #232]	(ec <CAN_Transmit+0xec>)
D:\STM32\Program\1.11_Odchudzanie\um0427\FWLib\library\src/stm32f10x_can.c:407
   2:	b510      	push	{r4, lr}
D:\STM32\Program\1.11_Odchudzanie\um0427\FWLib\library\src/stm32f10x_can.c:418
   4:	6893      	ldr	r3, [r2, #8]
D:\STM32\Program\1.11_Odchudzanie\um0427\FWLib\library\src/stm32f10x_can.c:407
   6:	4604      	mov	r4, r0
D:\STM32\Program\1.11_Odchudzanie\um0427\FWLib\library\src/stm32f10x_can.c:418
   8:	f013 6f80 	tst.w	r3, #67108864	; 0x4000000
   c:	d002      	beq.n	14 <CAN_Transmit+0x14>
   e:	f04f 0c00 	mov.w	ip, #0	; 0x0
  12:	e00f      	b.n	34 <CAN_Transmit+0x34>
D:\STM32\Program\1.11_Odchudzanie\um0427\FWLib\library\src/stm32f10x_can.c:422
  14:	6893      	ldr	r3, [r2, #8]
  16:	f013 6f00 	tst.w	r3, #134217728	; 0x8000000
  1a:	d002      	beq.n	22 <CAN_Transmit+0x22>
  1c:	f04f 0c01 	mov.w	ip, #1	; 0x1
  20:	e008      	b.n	34 <CAN_Transmit+0x34>
D:\STM32\Program\1.11_Odchudzanie\um0427\FWLib\library\src/stm32f10x_can.c:426
  22:	6893      	ldr	r3, [r2, #8]
  24:	f013 5f80 	tst.w	r3, #268435456	; 0x10000000
  28:	d102      	bne.n	30 <CAN_Transmit+0x30>
  2a:	f04f 0c04 	mov.w	ip, #4	; 0x4
  2e:	e05a      	b.n	e6 <CAN_Transmit+0xe6>
  30:	f04f 0c02 	mov.w	ip, #2	; 0x2
D:\STM32\Program\1.11_Odchudzanie\um0427\FWLib\library\src/stm32f10x_can.c:438
  34:	ea4f 130c 	mov.w	r3, ip, lsl #4
  38:	f103 4080 	add.w	r0, r3, #1073741824	; 0x40000000
  3c:	f500 40c8 	add.w	r0, r0, #25600	; 0x6400
  40:	f8d0 3180 	ldr.w	r3, [r0, #384]
  44:	f003 0301 	and.w	r3, r3, #1	; 0x1
  48:	f8c0 3180 	str.w	r3, [r0, #384]
D:\STM32\Program\1.11_Odchudzanie\um0427\FWLib\library\src/stm32f10x_can.c:439
  4c:	7a22      	ldrb	r2, [r4, #8]
  4e:	f894 e009 	ldrb.w	lr, [r4, #9]
  52:	b952      	cbnz	r2, 6a <CAN_Transmit+0x6a>
D:\STM32\Program\1.11_Odchudzanie\um0427\FWLib\library\src/stm32f10x_can.c:441
  54:	6822      	ldr	r2, [r4, #0]
D:\STM32\Program\1.11_Odchudzanie\um0427\FWLib\library\src/stm32f10x_can.c:442
  56:	0552      	lsls	r2, r2, #21
  58:	6022      	str	r2, [r4, #0]
D:\STM32\Program\1.11_Odchudzanie\um0427\FWLib\library\src/stm32f10x_can.c:444
  5a:	f8d0 3180 	ldr.w	r3, [r0, #384]
  5e:	ea4e 0303 	orr.w	r3, lr, r3
  62:	4313      	orrs	r3, r2
  64:	f8c0 3180 	str.w	r3, [r0, #384]
  68:	e00a      	b.n	80 <CAN_Transmit+0x80>
D:\STM32\Program\1.11_Odchudzanie\um0427\FWLib\library\src/stm32f10x_can.c:449
  6a:	6863      	ldr	r3, [r4, #4]
D:\STM32\Program\1.11_Odchudzanie\um0427\FWLib\library\src/stm32f10x_can.c:452
  6c:	ea42 020e 	orr.w	r2, r2, lr
D:\STM32\Program\1.11_Odchudzanie\um0427\FWLib\library\src/stm32f10x_can.c:450
  70:	00db      	lsls	r3, r3, #3
  72:	6063      	str	r3, [r4, #4]
D:\STM32\Program\1.11_Odchudzanie\um0427\FWLib\library\src/stm32f10x_can.c:452
  74:	f8d0 1180 	ldr.w	r1, [r0, #384]
  78:	430a      	orrs	r2, r1
  7a:	431a      	orrs	r2, r3
  7c:	f8c0 2180 	str.w	r2, [r0, #384]
D:\STM32\Program\1.11_Odchudzanie\um0427\FWLib\library\src/stm32f10x_can.c:457
  80:	7aa2      	ldrb	r2, [r4, #10]
D:\STM32\Program\1.11_Odchudzanie\um0427\FWLib\library\src/stm32f10x_can.c:458
  82:	ea4f 110c 	mov.w	r1, ip, lsl #4
D:\STM32\Program\1.11_Odchudzanie\um0427\FWLib\library\src/stm32f10x_can.c:457
  86:	f002 020f 	and.w	r2, r2, #15	; 0xf
D:\STM32\Program\1.11_Odchudzanie\um0427\FWLib\library\src/stm32f10x_can.c:458
  8a:	f101 4180 	add.w	r1, r1, #1073741824	; 0x40000000
D:\STM32\Program\1.11_Odchudzanie\um0427\FWLib\library\src/stm32f10x_can.c:457
  8e:	72a2      	strb	r2, [r4, #10]
D:\STM32\Program\1.11_Odchudzanie\um0427\FWLib\library\src/stm32f10x_can.c:458
  90:	f501 41c8 	add.w	r1, r1, #25600	; 0x6400
  94:	f8d1 3184 	ldr.w	r3, [r1, #388]
  98:	f023 030f 	bic.w	r3, r3, #15	; 0xf
  9c:	f8c1 3184 	str.w	r3, [r1, #388]
D:\STM32\Program\1.11_Odchudzanie\um0427\FWLib\library\src/stm32f10x_can.c:459
  a0:	f8d1 3184 	ldr.w	r3, [r1, #388]
  a4:	431a      	orrs	r2, r3
  a6:	f8c1 2184 	str.w	r2, [r1, #388]
D:\STM32\Program\1.11_Odchudzanie\um0427\FWLib\library\src/stm32f10x_can.c:462
  aa:	7b63      	ldrb	r3, [r4, #13]
  ac:	7ba2      	ldrb	r2, [r4, #14]
  ae:	041b      	lsls	r3, r3, #16
  b0:	ea43 6302 	orr.w	r3, r3, r2, lsl #24
  b4:	7ae2      	ldrb	r2, [r4, #11]
  b6:	4313      	orrs	r3, r2
  b8:	7b22      	ldrb	r2, [r4, #12]
  ba:	ea43 2302 	orr.w	r3, r3, r2, lsl #8
  be:	f8c1 3188 	str.w	r3, [r1, #392]
D:\STM32\Program\1.11_Odchudzanie\um0427\FWLib\library\src/stm32f10x_can.c:466
  c2:	7c63      	ldrb	r3, [r4, #17]
  c4:	7ca2      	ldrb	r2, [r4, #18]
  c6:	041b      	lsls	r3, r3, #16
  c8:	ea43 6302 	orr.w	r3, r3, r2, lsl #24
  cc:	7be2      	ldrb	r2, [r4, #15]
  ce:	4313      	orrs	r3, r2
  d0:	7c22      	ldrb	r2, [r4, #16]
  d2:	ea43 2302 	orr.w	r3, r3, r2, lsl #8
  d6:	f8c1 318c 	str.w	r3, [r1, #396]
D:\STM32\Program\1.11_Odchudzanie\um0427\FWLib\library\src/stm32f10x_can.c:472
  da:	f8d1 3180 	ldr.w	r3, [r1, #384]
  de:	f043 0301 	orr.w	r3, r3, #1	; 0x1
  e2:	f8c1 3180 	str.w	r3, [r1, #384]
D:\STM32\Program\1.11_Odchudzanie\um0427\FWLib\library\src/stm32f10x_can.c:476
  e6:	4660      	mov	r0, ip
  e8:	bd10      	pop	{r4, pc}
  ea:	46c0      	nop			(mov r8, r8)
  ec:	40006400 	.word	0x40006400
Disassembly of section .text.CAN_TransmitStatus:

00000000 <CAN_TransmitStatus>:
CAN_TransmitStatus():
D:\STM32\Program\1.11_Odchudzanie\um0427\FWLib\library\src/stm32f10x_can.c:495
   0:	2801      	cmp	r0, #1
   2:	d010      	beq.n	26 <CAN_TransmitStatus+0x26>
   4:	d302      	bcc.n	c <CAN_TransmitStatus+0xc>
   6:	2802      	cmp	r0, #2
   8:	d01b      	beq.n	42 <CAN_TransmitStatus+0x42>
   a:	e02f      	b.n	6c <CAN_TransmitStatus+0x6c>
D:\STM32\Program\1.11_Odchudzanie\um0427\FWLib\library\src/stm32f10x_can.c:497
   c:	4918      	ldr	r1, [pc, #96]	(70 <CAN_TransmitStatus+0x70>)
   e:	688b      	ldr	r3, [r1, #8]
D:\STM32\Program\1.11_Odchudzanie\um0427\FWLib\library\src/stm32f10x_can.c:498
  10:	688a      	ldr	r2, [r1, #8]
  12:	f003 0301 	and.w	r3, r3, #1	; 0x1
  16:	f002 0202 	and.w	r2, r2, #2	; 0x2
  1a:	ea42 0283 	orr.w	r2, r2, r3, lsl #2
D:\STM32\Program\1.11_Odchudzanie\um0427\FWLib\library\src/stm32f10x_can.c:499
  1e:	688b      	ldr	r3, [r1, #8]
  20:	f3c3 6380 	ubfx	r3, r3, #26, #1
  24:	e01a      	b.n	5c <CAN_TransmitStatus+0x5c>
D:\STM32\Program\1.11_Odchudzanie\um0427\FWLib\library\src/stm32f10x_can.c:501
  26:	4a12      	ldr	r2, [pc, #72]	(70 <CAN_TransmitStatus+0x70>)
  28:	6893      	ldr	r3, [r2, #8]
D:\STM32\Program\1.11_Odchudzanie\um0427\FWLib\library\src/stm32f10x_can.c:502
  2a:	6891      	ldr	r1, [r2, #8]
  2c:	f403 7380 	and.w	r3, r3, #256	; 0x100
D:\STM32\Program\1.11_Odchudzanie\um0427\FWLib\library\src/stm32f10x_can.c:503
  30:	6892      	ldr	r2, [r2, #8]
D:\STM32\Program\1.11_Odchudzanie\um0427\FWLib\library\src/stm32f10x_can.c:502
  32:	f401 7100 	and.w	r1, r1, #512	; 0x200
  36:	099b      	lsrs	r3, r3, #6
  38:	ea43 2311 	orr.w	r3, r3, r1, lsr #8
D:\STM32\Program\1.11_Odchudzanie\um0427\FWLib\library\src/stm32f10x_can.c:503
  3c:	f3c2 62c0 	ubfx	r2, r2, #27, #1
  40:	e00c      	b.n	5c <CAN_TransmitStatus+0x5c>
D:\STM32\Program\1.11_Odchudzanie\um0427\FWLib\library\src/stm32f10x_can.c:505
  42:	4a0b      	ldr	r2, [pc, #44]	(70 <CAN_TransmitStatus+0x70>)
  44:	6893      	ldr	r3, [r2, #8]
D:\STM32\Program\1.11_Odchudzanie\um0427\FWLib\library\src/stm32f10x_can.c:506
  46:	6891      	ldr	r1, [r2, #8]
  48:	f403 3380 	and.w	r3, r3, #65536	; 0x10000
D:\STM32\Program\1.11_Odchudzanie\um0427\FWLib\library\src/stm32f10x_can.c:507
  4c:	6892      	ldr	r2, [r2, #8]
D:\STM32\Program\1.11_Odchudzanie\um0427\FWLib\library\src/stm32f10x_can.c:506
  4e:	f401 3100 	and.w	r1, r1, #131072	; 0x20000
  52:	0b9b      	lsrs	r3, r3, #14
  54:	ea43 4311 	orr.w	r3, r3, r1, lsr #16
D:\STM32\Program\1.11_Odchudzanie\um0427\FWLib\library\src/stm32f10x_can.c:507
  58:	f3c2 7200 	ubfx	r2, r2, #28, #1
  5c:	ea43 0002 	orr.w	r0, r3, r2
D:\STM32\Program\1.11_Odchudzanie\um0427\FWLib\library\src/stm32f10x_can.c:514
  60:	b120      	cbz	r0, 6c <CAN_TransmitStatus+0x6c>
  62:	2807      	cmp	r0, #7
  64:	bf14      	ite	ne
  66:	2000      	movne	r0, #0
  68:	2001      	moveq	r0, #1
  6a:	e000      	b.n	6e <CAN_TransmitStatus+0x6e>
  6c:	2002      	movs	r0, #2
D:\STM32\Program\1.11_Odchudzanie\um0427\FWLib\library\src/stm32f10x_can.c:531
  6e:	4770      	bx	lr
  70:	40006400 	.word	0x40006400
Disassembly of section .text.CAN_CancelTransmit:

00000000 <CAN_CancelTransmit>:
CAN_CancelTransmit():
D:\STM32\Program\1.11_Odchudzanie\um0427\FWLib\library\src/stm32f10x_can.c:546
   0:	2801      	cmp	r0, #1
   2:	d008      	beq.n	16 <CAN_CancelTransmit+0x16>
   4:	d302      	bcc.n	c <CAN_CancelTransmit+0xc>
   6:	2802      	cmp	r0, #2
   8:	d00a      	beq.n	20 <CAN_CancelTransmit+0x20>
   a:	e00e      	b.n	2a <CAN_CancelTransmit+0x2a>
D:\STM32\Program\1.11_Odchudzanie\um0427\FWLib\library\src/stm32f10x_can.c:548
   c:	4a07      	ldr	r2, [pc, #28]	(2c <CAN_CancelTransmit+0x2c>)
   e:	6893      	ldr	r3, [r2, #8]
  10:	f043 0380 	orr.w	r3, r3, #128	; 0x80
  14:	e008      	b.n	28 <CAN_CancelTransmit+0x28>
D:\STM32\Program\1.11_Odchudzanie\um0427\FWLib\library\src/stm32f10x_can.c:550
  16:	4a05      	ldr	r2, [pc, #20]	(2c <CAN_CancelTransmit+0x2c>)
  18:	6893      	ldr	r3, [r2, #8]
  1a:	f443 4300 	orr.w	r3, r3, #32768	; 0x8000
  1e:	e003      	b.n	28 <CAN_CancelTransmit+0x28>
D:\STM32\Program\1.11_Odchudzanie\um0427\FWLib\library\src/stm32f10x_can.c:552
  20:	4a02      	ldr	r2, [pc, #8]	(2c <CAN_CancelTransmit+0x2c>)
  22:	6893      	ldr	r3, [r2, #8]
  24:	f443 0300 	orr.w	r3, r3, #8388608	; 0x800000
  28:	6093      	str	r3, [r2, #8]
D:\STM32\Program\1.11_Odchudzanie\um0427\FWLib\library\src/stm32f10x_can.c:557
  2a:	4770      	bx	lr
  2c:	40006400 	.word	0x40006400
Disassembly of section .text.CAN_FIFORelease:

00000000 <CAN_FIFORelease>:
CAN_FIFORelease():
D:\STM32\Program\1.11_Odchudzanie\um0427\FWLib\library\src/stm32f10x_can.c:572
   0:	b918      	cbnz	r0, a <CAN_FIFORelease+0xa>
D:\STM32\Program\1.11_Odchudzanie\um0427\FWLib\library\src/stm32f10x_can.c:574
   2:	4b04      	ldr	r3, [pc, #16]	(14 <CAN_FIFORelease+0x14>)
   4:	2220      	movs	r2, #32
   6:	60da      	str	r2, [r3, #12]
   8:	e002      	b.n	10 <CAN_FIFORelease+0x10>
D:\STM32\Program\1.11_Odchudzanie\um0427\FWLib\library\src/stm32f10x_can.c:579
   a:	4b02      	ldr	r3, [pc, #8]	(14 <CAN_FIFORelease+0x14>)
   c:	2220      	movs	r2, #32
   e:	611a      	str	r2, [r3, #16]
D:\STM32\Program\1.11_Odchudzanie\um0427\FWLib\library\src/stm32f10x_can.c:581
  10:	4770      	bx	lr
  12:	46c0      	nop			(mov r8, r8)
  14:	40006400 	.word	0x40006400
Disassembly of section .text.CAN_MessagePending:

00000000 <CAN_MessagePending>:
CAN_MessagePending():
D:\STM32\Program\1.11_Odchudzanie\um0427\FWLib\library\src/stm32f10x_can.c:597
   0:	b910      	cbnz	r0, 8 <CAN_MessagePending+0x8>
D:\STM32\Program\1.11_Odchudzanie\um0427\FWLib\library\src/stm32f10x_can.c:599
   2:	4b06      	ldr	r3, [pc, #24]	(1c <CAN_MessagePending+0x1c>)
   4:	68db      	ldr	r3, [r3, #12]
   6:	e005      	b.n	14 <CAN_MessagePending+0x14>
D:\STM32\Program\1.11_Odchudzanie\um0427\FWLib\library\src/stm32f10x_can.c:601
   8:	2801      	cmp	r0, #1
   a:	d001      	beq.n	10 <CAN_MessagePending+0x10>
   c:	2000      	movs	r0, #0
   e:	e003      	b.n	18 <CAN_MessagePending+0x18>
D:\STM32\Program\1.11_Odchudzanie\um0427\FWLib\library\src/stm32f10x_can.c:603
  10:	4b02      	ldr	r3, [pc, #8]	(1c <CAN_MessagePending+0x1c>)
  12:	691b      	ldr	r3, [r3, #16]
  14:	f003 0003 	and.w	r0, r3, #3	; 0x3
D:\STM32\Program\1.11_Odchudzanie\um0427\FWLib\library\src/stm32f10x_can.c:610
  18:	4770      	bx	lr
  1a:	46c0      	nop			(mov r8, r8)
  1c:	40006400 	.word	0x40006400
Disassembly of section .text.CAN_Receive:

00000000 <CAN_Receive>:
CAN_Receive():
D:\STM32\Program\1.11_Odchudzanie\um0427\FWLib\library\src/stm32f10x_can.c:626
   0:	0103      	lsls	r3, r0, #4
   2:	f103 4280 	add.w	r2, r3, #1073741824	; 0x40000000
   6:	f502 42c8 	add.w	r2, r2, #25600	; 0x6400
   a:	f8d2 31b0 	ldr.w	r3, [r2, #432]
D:\STM32\Program\1.11_Odchudzanie\um0427\FWLib\library\src/stm32f10x_can.c:621
   e:	b510      	push	{r4, lr}
D:\STM32\Program\1.11_Odchudzanie\um0427\FWLib\library\src/stm32f10x_can.c:626
  10:	f003 0304 	and.w	r3, r3, #4	; 0x4
  14:	720b      	strb	r3, [r1, #8]
D:\STM32\Program\1.11_Odchudzanie\um0427\FWLib\library\src/stm32f10x_can.c:627
  16:	b923      	cbnz	r3, 22 <CAN_Receive+0x22>
D:\STM32\Program\1.11_Odchudzanie\um0427\FWLib\library\src/stm32f10x_can.c:629
  18:	f8d2 31b0 	ldr.w	r3, [r2, #432]
  1c:	0d5b      	lsrs	r3, r3, #21
  1e:	600b      	str	r3, [r1, #0]
  20:	e003      	b.n	2a <CAN_Receive+0x2a>
D:\STM32\Program\1.11_Odchudzanie\um0427\FWLib\library\src/stm32f10x_can.c:633
  22:	f8d2 31b0 	ldr.w	r3, [r2, #432]
  26:	08db      	lsrs	r3, r3, #3
  28:	604b      	str	r3, [r1, #4]
D:\STM32\Program\1.11_Odchudzanie\um0427\FWLib\library\src/stm32f10x_can.c:636
  2a:	0102      	lsls	r2, r0, #4
  2c:	f102 4280 	add.w	r2, r2, #1073741824	; 0x40000000
  30:	f502 42c8 	add.w	r2, r2, #25600	; 0x6400
  34:	f8d2 31b0 	ldr.w	r3, [r2, #432]
  38:	f003 0302 	and.w	r3, r3, #2	; 0x2
  3c:	724b      	strb	r3, [r1, #9]
D:\STM32\Program\1.11_Odchudzanie\um0427\FWLib\library\src/stm32f10x_can.c:639
  3e:	f8d2 31b4 	ldr.w	r3, [r2, #436]
  42:	f003 030f 	and.w	r3, r3, #15	; 0xf
  46:	728b      	strb	r3, [r1, #10]
D:\STM32\Program\1.11_Odchudzanie\um0427\FWLib\library\src/stm32f10x_can.c:642
  48:	f8d2 31b4 	ldr.w	r3, [r2, #436]
  4c:	0a1b      	lsrs	r3, r3, #8
  4e:	74cb      	strb	r3, [r1, #19]
D:\STM32\Program\1.11_Odchudzanie\um0427\FWLib\library\src/stm32f10x_can.c:645
  50:	f8d2 31b8 	ldr.w	r3, [r2, #440]
  54:	72cb      	strb	r3, [r1, #11]
D:\STM32\Program\1.11_Odchudzanie\um0427\FWLib\library\src/stm32f10x_can.c:646
  56:	f8d2 31b8 	ldr.w	r3, [r2, #440]
  5a:	0a1b      	lsrs	r3, r3, #8
  5c:	730b      	strb	r3, [r1, #12]
D:\STM32\Program\1.11_Odchudzanie\um0427\FWLib\library\src/stm32f10x_can.c:647
  5e:	f8d2 31b8 	ldr.w	r3, [r2, #440]
  62:	0c1b      	lsrs	r3, r3, #16
  64:	734b      	strb	r3, [r1, #13]
D:\STM32\Program\1.11_Odchudzanie\um0427\FWLib\library\src/stm32f10x_can.c:648
  66:	f8d2 31b8 	ldr.w	r3, [r2, #440]
  6a:	0e1b      	lsrs	r3, r3, #24
  6c:	738b      	strb	r3, [r1, #14]
D:\STM32\Program\1.11_Odchudzanie\um0427\FWLib\library\src/stm32f10x_can.c:650
  6e:	f8d2 31bc 	ldr.w	r3, [r2, #444]
  72:	73cb      	strb	r3, [r1, #15]
D:\STM32\Program\1.11_Odchudzanie\um0427\FWLib\library\src/stm32f10x_can.c:651
  74:	f8d2 31bc 	ldr.w	r3, [r2, #444]
  78:	0a1b      	lsrs	r3, r3, #8
  7a:	740b      	strb	r3, [r1, #16]
D:\STM32\Program\1.11_Odchudzanie\um0427\FWLib\library\src/stm32f10x_can.c:652
  7c:	f8d2 31bc 	ldr.w	r3, [r2, #444]
  80:	0c1b      	lsrs	r3, r3, #16
  82:	744b      	strb	r3, [r1, #17]
D:\STM32\Program\1.11_Odchudzanie\um0427\FWLib\library\src/stm32f10x_can.c:653
  84:	f8d2 31bc 	ldr.w	r3, [r2, #444]
  88:	0e1b      	lsrs	r3, r3, #24
  8a:	748b      	strb	r3, [r1, #18]
D:\STM32\Program\1.11_Odchudzanie\um0427\FWLib\library\src/stm32f10x_can.c:656
  8c:	f7ff fffe 	bl	0 <CAN_Receive>
D:\STM32\Program\1.11_Odchudzanie\um0427\FWLib\library\src/stm32f10x_can.c:657
  90:	bd10      	pop	{r4, pc}
  92:	46c0      	nop			(mov r8, r8)
Disassembly of section .text.CAN_Sleep:

00000000 <CAN_Sleep>:
CAN_Sleep():
D:\STM32\Program\1.11_Odchudzanie\um0427\FWLib\library\src/stm32f10x_can.c:671
   0:	4b04      	ldr	r3, [pc, #16]	(14 <CAN_Sleep+0x14>)
   2:	681a      	ldr	r2, [r3, #0]
   4:	f042 0202 	orr.w	r2, r2, #2	; 0x2
   8:	601a      	str	r2, [r3, #0]
D:\STM32\Program\1.11_Odchudzanie\um0427\FWLib\library\src/stm32f10x_can.c:675
   a:	6818      	ldr	r0, [r3, #0]
D:\STM32\Program\1.11_Odchudzanie\um0427\FWLib\library\src/stm32f10x_can.c:683
   c:	f3c0 0040 	ubfx	r0, r0, #1, #1
  10:	4770      	bx	lr
  12:	46c0      	nop			(mov r8, r8)
  14:	40006400 	.word	0x40006400
Disassembly of section .text.CAN_WakeUp:

00000000 <CAN_WakeUp>:
CAN_WakeUp():
D:\STM32\Program\1.11_Odchudzanie\um0427\FWLib\library\src/stm32f10x_can.c:698
   0:	4b05      	ldr	r3, [pc, #20]	(18 <CAN_WakeUp+0x18>)
   2:	681a      	ldr	r2, [r3, #0]
   4:	f022 0202 	bic.w	r2, r2, #2	; 0x2
   8:	601a      	str	r2, [r3, #0]
D:\STM32\Program\1.11_Odchudzanie\um0427\FWLib\library\src/stm32f10x_can.c:702
   a:	6818      	ldr	r0, [r3, #0]
   c:	f080 0002 	eor.w	r0, r0, #2	; 0x2
D:\STM32\Program\1.11_Odchudzanie\um0427\FWLib\library\src/stm32f10x_can.c:710
  10:	f3c0 0040 	ubfx	r0, r0, #1, #1
  14:	4770      	bx	lr
  16:	46c0      	nop			(mov r8, r8)
  18:	40006400 	.word	0x40006400
Disassembly of section .text.CAN_GetFlagStatus:

00000000 <CAN_GetFlagStatus>:
CAN_GetFlagStatus():
D:\STM32\Program\1.11_Odchudzanie\um0427\FWLib\library\src/stm32f10x_can.c:729
   0:	4b03      	ldr	r3, [pc, #12]	(10 <CAN_GetFlagStatus+0x10>)
   2:	699b      	ldr	r3, [r3, #24]
   4:	4218      	tst	r0, r3
D:\STM32\Program\1.11_Odchudzanie\um0427\FWLib\library\src/stm32f10x_can.c:741
   6:	bf0c      	ite	eq
   8:	2000      	moveq	r0, #0
   a:	2001      	movne	r0, #1
   c:	4770      	bx	lr
   e:	46c0      	nop			(mov r8, r8)
  10:	40006400 	.word	0x40006400
Disassembly of section .text.CAN_ClearFlag:

00000000 <CAN_ClearFlag>:
CAN_ClearFlag():
D:\STM32\Program\1.11_Odchudzanie\um0427\FWLib\library\src/stm32f10x_can.c:756
   0:	4a02      	ldr	r2, [pc, #8]	(c <CAN_ClearFlag+0xc>)
   2:	6993      	ldr	r3, [r2, #24]
   4:	ea23 0300 	bic.w	r3, r3, r0
   8:	6193      	str	r3, [r2, #24]
D:\STM32\Program\1.11_Odchudzanie\um0427\FWLib\library\src/stm32f10x_can.c:757
   a:	4770      	bx	lr
   c:	40006400 	.word	0x40006400
Disassembly of section .text.CAN_ClearITPendingBit:

00000000 <CAN_ClearITPendingBit>:
CAN_ClearITPendingBit():
D:\STM32\Program\1.11_Odchudzanie\um0427\FWLib\library\src/stm32f10x_can.c:838
   0:	2820      	cmp	r0, #32
   2:	d031      	beq.n	68 <CAN_ClearITPendingBit+0x68>
   4:	d80c      	bhi.n	20 <CAN_ClearITPendingBit+0x20>
   6:	2806      	cmp	r0, #6
   8:	d020      	beq.n	4c <CAN_ClearITPendingBit+0x4c>
   a:	d804      	bhi.n	16 <CAN_ClearITPendingBit+0x16>
   c:	2804      	cmp	r0, #4
   e:	d025      	beq.n	5c <CAN_ClearITPendingBit+0x5c>
  10:	2805      	cmp	r0, #5
  12:	d019      	beq.n	48 <CAN_ClearITPendingBit+0x48>
  14:	e043      	b.n	9e <CAN_ClearITPendingBit+0x9e>
  16:	2807      	cmp	r0, #7
  18:	d01d      	beq.n	56 <CAN_ClearITPendingBit+0x56>
  1a:	2808      	cmp	r0, #8
  1c:	d020      	beq.n	60 <CAN_ClearITPendingBit+0x60>
  1e:	e03e      	b.n	9e <CAN_ClearITPendingBit+0x9e>
  20:	f5b0 7f00 	cmp.w	r0, #512	; 0x200
  24:	d02b      	beq.n	7e <CAN_ClearITPendingBit+0x7e>
  26:	d805      	bhi.n	34 <CAN_ClearITPendingBit+0x34>
  28:	2840      	cmp	r0, #64
  2a:	d01f      	beq.n	6c <CAN_ClearITPendingBit+0x6c>
  2c:	f5b0 7f80 	cmp.w	r0, #256	; 0x100
  30:	d020      	beq.n	74 <CAN_ClearITPendingBit+0x74>
  32:	e034      	b.n	9e <CAN_ClearITPendingBit+0x9e>
  34:	f5b0 3f80 	cmp.w	r0, #65536	; 0x10000
  38:	d02c      	beq.n	94 <CAN_ClearITPendingBit+0x94>
  3a:	f5b0 3f00 	cmp.w	r0, #131072	; 0x20000
  3e:	d02b      	beq.n	98 <CAN_ClearITPendingBit+0x98>
  40:	f5b0 6f80 	cmp.w	r0, #1024	; 0x400
  44:	d020      	beq.n	88 <CAN_ClearITPendingBit+0x88>
  46:	e02a      	b.n	9e <CAN_ClearITPendingBit+0x9e>
D:\STM32\Program\1.11_Odchudzanie\um0427\FWLib\library\src/stm32f10x_can.c:841
  48:	2201      	movs	r2, #1
  4a:	e001      	b.n	50 <CAN_ClearITPendingBit+0x50>
D:\STM32\Program\1.11_Odchudzanie\um0427\FWLib\library\src/stm32f10x_can.c:844
  4c:	f44f 7280 	mov.w	r2, #256	; 0x100
  50:	4b13      	ldr	r3, [pc, #76]	(a0 <CAN_ClearITPendingBit+0xa0>)
  52:	609a      	str	r2, [r3, #8]
D:\STM32\Program\1.11_Odchudzanie\um0427\FWLib\library\src/stm32f10x_can.c:845
  54:	e023      	b.n	9e <CAN_ClearITPendingBit+0x9e>
D:\STM32\Program\1.11_Odchudzanie\um0427\FWLib\library\src/stm32f10x_can.c:847
  56:	f44f 3280 	mov.w	r2, #65536	; 0x10000
  5a:	e7f9      	b.n	50 <CAN_ClearITPendingBit+0x50>
D:\STM32\Program\1.11_Odchudzanie\um0427\FWLib\library\src/stm32f10x_can.c:850
  5c:	2208      	movs	r2, #8
  5e:	e000      	b.n	62 <CAN_ClearITPendingBit+0x62>
D:\STM32\Program\1.11_Odchudzanie\um0427\FWLib\library\src/stm32f10x_can.c:853
  60:	2210      	movs	r2, #16
  62:	4b0f      	ldr	r3, [pc, #60]	(a0 <CAN_ClearITPendingBit+0xa0>)
  64:	60da      	str	r2, [r3, #12]
D:\STM32\Program\1.11_Odchudzanie\um0427\FWLib\library\src/stm32f10x_can.c:854
  66:	e01a      	b.n	9e <CAN_ClearITPendingBit+0x9e>
D:\STM32\Program\1.11_Odchudzanie\um0427\FWLib\library\src/stm32f10x_can.c:856
  68:	2208      	movs	r2, #8
  6a:	e000      	b.n	6e <CAN_ClearITPendingBit+0x6e>
D:\STM32\Program\1.11_Odchudzanie\um0427\FWLib\library\src/stm32f10x_can.c:859
  6c:	2210      	movs	r2, #16
  6e:	4b0c      	ldr	r3, [pc, #48]	(a0 <CAN_ClearITPendingBit+0xa0>)
  70:	611a      	str	r2, [r3, #16]
D:\STM32\Program\1.11_Odchudzanie\um0427\FWLib\library\src/stm32f10x_can.c:860
  72:	e014      	b.n	9e <CAN_ClearITPendingBit+0x9e>
D:\STM32\Program\1.11_Odchudzanie\um0427\FWLib\library\src/stm32f10x_can.c:862
  74:	4a0a      	ldr	r2, [pc, #40]	(a0 <CAN_ClearITPendingBit+0xa0>)
  76:	6993      	ldr	r3, [r2, #24]
  78:	f023 0301 	bic.w	r3, r3, #1	; 0x1
  7c:	e008      	b.n	90 <CAN_ClearITPendingBit+0x90>
D:\STM32\Program\1.11_Odchudzanie\um0427\FWLib\library\src/stm32f10x_can.c:865
  7e:	4a08      	ldr	r2, [pc, #32]	(a0 <CAN_ClearITPendingBit+0xa0>)
  80:	6993      	ldr	r3, [r2, #24]
  82:	f023 0302 	bic.w	r3, r3, #2	; 0x2
  86:	e003      	b.n	90 <CAN_ClearITPendingBit+0x90>
D:\STM32\Program\1.11_Odchudzanie\um0427\FWLib\library\src/stm32f10x_can.c:868
  88:	4a05      	ldr	r2, [pc, #20]	(a0 <CAN_ClearITPendingBit+0xa0>)
  8a:	6993      	ldr	r3, [r2, #24]
  8c:	f023 0304 	bic.w	r3, r3, #4	; 0x4
  90:	6193      	str	r3, [r2, #24]
D:\STM32\Program\1.11_Odchudzanie\um0427\FWLib\library\src/stm32f10x_can.c:869
  92:	e004      	b.n	9e <CAN_ClearITPendingBit+0x9e>
D:\STM32\Program\1.11_Odchudzanie\um0427\FWLib\library\src/stm32f10x_can.c:871
  94:	2208      	movs	r2, #8
  96:	e000      	b.n	9a <CAN_ClearITPendingBit+0x9a>
D:\STM32\Program\1.11_Odchudzanie\um0427\FWLib\library\src/stm32f10x_can.c:874
  98:	2210      	movs	r2, #16
  9a:	4b01      	ldr	r3, [pc, #4]	(a0 <CAN_ClearITPendingBit+0xa0>)
  9c:	605a      	str	r2, [r3, #4]
D:\STM32\Program\1.11_Odchudzanie\um0427\FWLib\library\src/stm32f10x_can.c:879
  9e:	4770      	bx	lr
  a0:	40006400 	.word	0x40006400
Disassembly of section .text.CheckITStatus:

00000000 <CheckITStatus>:
CheckITStatus():
D:\STM32\Program\1.11_Odchudzanie\um0427\FWLib\library\src/stm32f10x_can.c:890
   0:	4201      	tst	r1, r0
D:\STM32\Program\1.11_Odchudzanie\um0427\FWLib\library\src/stm32f10x_can.c:905
   2:	bf0c      	ite	eq
   4:	2000      	moveq	r0, #0
   6:	2001      	movne	r0, #1
   8:	4770      	bx	lr
   a:	46c0      	nop			(mov r8, r8)
Disassembly of section .text.CAN_GetITStatus:

00000000 <CAN_GetITStatus>:
CAN_GetITStatus():
D:\STM32\Program\1.11_Odchudzanie\um0427\FWLib\library\src/stm32f10x_can.c:778
   0:	2820      	cmp	r0, #32
D:\STM32\Program\1.11_Odchudzanie\um0427\FWLib\library\src/stm32f10x_can.c:772
   2:	b510      	push	{r4, lr}
D:\STM32\Program\1.11_Odchudzanie\um0427\FWLib\library\src/stm32f10x_can.c:778
   4:	d035      	beq.n	72 <CAN_GetITStatus+0x72>
   6:	d80c      	bhi.n	22 <CAN_GetITStatus+0x22>
   8:	2806      	cmp	r0, #6
   a:	d022      	beq.n	52 <CAN_GetITStatus+0x52>
   c:	d804      	bhi.n	18 <CAN_GetITStatus+0x18>
   e:	2804      	cmp	r0, #4
  10:	d029      	beq.n	66 <CAN_GetITStatus+0x66>
  12:	2805      	cmp	r0, #5
  14:	d01a      	beq.n	4c <CAN_GetITStatus+0x4c>
  16:	e017      	b.n	48 <CAN_GetITStatus+0x48>
  18:	2807      	cmp	r0, #7
  1a:	d01f      	beq.n	5c <CAN_GetITStatus+0x5c>
  1c:	2808      	cmp	r0, #8
  1e:	d025      	beq.n	6c <CAN_GetITStatus+0x6c>
  20:	e012      	b.n	48 <CAN_GetITStatus+0x48>
  22:	f5b0 7f00 	cmp.w	r0, #512	; 0x200
  26:	d02e      	beq.n	86 <CAN_GetITStatus+0x86>
  28:	d805      	bhi.n	36 <CAN_GetITStatus+0x36>
  2a:	2840      	cmp	r0, #64
  2c:	d024      	beq.n	78 <CAN_GetITStatus+0x78>
  2e:	f5b0 7f80 	cmp.w	r0, #256	; 0x100
  32:	d024      	beq.n	7e <CAN_GetITStatus+0x7e>
  34:	e008      	b.n	48 <CAN_GetITStatus+0x48>
  36:	f5b0 3f80 	cmp.w	r0, #65536	; 0x10000
  3a:	d030      	beq.n	9e <CAN_GetITStatus+0x9e>
  3c:	f5b0 3f00 	cmp.w	r0, #131072	; 0x20000
  40:	d029      	beq.n	96 <CAN_GetITStatus+0x96>
  42:	f5b0 6f80 	cmp.w	r0, #1024	; 0x400
  46:	d022      	beq.n	8e <CAN_GetITStatus+0x8e>
  48:	2000      	movs	r0, #0
  4a:	e02d      	b.n	a8 <CAN_GetITStatus+0xa8>
D:\STM32\Program\1.11_Odchudzanie\um0427\FWLib\library\src/stm32f10x_can.c:781
  4c:	4b17      	ldr	r3, [pc, #92]	(ac <CAN_GetITStatus+0xac>)
  4e:	6898      	ldr	r0, [r3, #8]
  50:	e017      	b.n	82 <CAN_GetITStatus+0x82>
D:\STM32\Program\1.11_Odchudzanie\um0427\FWLib\library\src/stm32f10x_can.c:784
  52:	4b16      	ldr	r3, [pc, #88]	(ac <CAN_GetITStatus+0xac>)
  54:	f44f 7180 	mov.w	r1, #256	; 0x100
  58:	6898      	ldr	r0, [r3, #8]
  5a:	e023      	b.n	a4 <CAN_GetITStatus+0xa4>
D:\STM32\Program\1.11_Odchudzanie\um0427\FWLib\library\src/stm32f10x_can.c:787
  5c:	4b13      	ldr	r3, [pc, #76]	(ac <CAN_GetITStatus+0xac>)
  5e:	f44f 3180 	mov.w	r1, #65536	; 0x10000
  62:	6898      	ldr	r0, [r3, #8]
  64:	e01e      	b.n	a4 <CAN_GetITStatus+0xa4>
D:\STM32\Program\1.11_Odchudzanie\um0427\FWLib\library\src/stm32f10x_can.c:790
  66:	4b11      	ldr	r3, [pc, #68]	(ac <CAN_GetITStatus+0xac>)
  68:	68d8      	ldr	r0, [r3, #12]
  6a:	e01a      	b.n	a2 <CAN_GetITStatus+0xa2>
D:\STM32\Program\1.11_Odchudzanie\um0427\FWLib\library\src/stm32f10x_can.c:793
  6c:	4b0f      	ldr	r3, [pc, #60]	(ac <CAN_GetITStatus+0xac>)
  6e:	68d8      	ldr	r0, [r3, #12]
  70:	e013      	b.n	9a <CAN_GetITStatus+0x9a>
D:\STM32\Program\1.11_Odchudzanie\um0427\FWLib\library\src/stm32f10x_can.c:796
  72:	4b0e      	ldr	r3, [pc, #56]	(ac <CAN_GetITStatus+0xac>)
  74:	6918      	ldr	r0, [r3, #16]
  76:	e014      	b.n	a2 <CAN_GetITStatus+0xa2>
D:\STM32\Program\1.11_Odchudzanie\um0427\FWLib\library\src/stm32f10x_can.c:799
  78:	4b0c      	ldr	r3, [pc, #48]	(ac <CAN_GetITStatus+0xac>)
  7a:	6918      	ldr	r0, [r3, #16]
  7c:	e00d      	b.n	9a <CAN_GetITStatus+0x9a>
D:\STM32\Program\1.11_Odchudzanie\um0427\FWLib\library\src/stm32f10x_can.c:802
  7e:	4b0b      	ldr	r3, [pc, #44]	(ac <CAN_GetITStatus+0xac>)
  80:	6998      	ldr	r0, [r3, #24]
  82:	2101      	movs	r1, #1
  84:	e00e      	b.n	a4 <CAN_GetITStatus+0xa4>
D:\STM32\Program\1.11_Odchudzanie\um0427\FWLib\library\src/stm32f10x_can.c:805
  86:	4b09      	ldr	r3, [pc, #36]	(ac <CAN_GetITStatus+0xac>)
  88:	2102      	movs	r1, #2
  8a:	6998      	ldr	r0, [r3, #24]
  8c:	e00a      	b.n	a4 <CAN_GetITStatus+0xa4>
D:\STM32\Program\1.11_Odchudzanie\um0427\FWLib\library\src/stm32f10x_can.c:808
  8e:	4b07      	ldr	r3, [pc, #28]	(ac <CAN_GetITStatus+0xac>)
  90:	2104      	movs	r1, #4
  92:	6998      	ldr	r0, [r3, #24]
  94:	e006      	b.n	a4 <CAN_GetITStatus+0xa4>
D:\STM32\Program\1.11_Odchudzanie\um0427\FWLib\library\src/stm32f10x_can.c:811
  96:	4b05      	ldr	r3, [pc, #20]	(ac <CAN_GetITStatus+0xac>)
  98:	6858      	ldr	r0, [r3, #4]
  9a:	2110      	movs	r1, #16
  9c:	e002      	b.n	a4 <CAN_GetITStatus+0xa4>
D:\STM32\Program\1.11_Odchudzanie\um0427\FWLib\library\src/stm32f10x_can.c:814
  9e:	4b03      	ldr	r3, [pc, #12]	(ac <CAN_GetITStatus+0xac>)
  a0:	6858      	ldr	r0, [r3, #4]
  a2:	2108      	movs	r1, #8
  a4:	f7ff fffe 	bl	0 <CAN_GetITStatus>
D:\STM32\Program\1.11_Odchudzanie\um0427\FWLib\library\src/stm32f10x_can.c:824
  a8:	bd10      	pop	{r4, pc}
  aa:	46c0      	nop			(mov r8, r8)
  ac:	40006400 	.word	0x40006400
Disassembly of section .text.CAN_DeInit:

00000000 <CAN_DeInit>:
CAN_DeInit():
D:\STM32\Program\1.11_Odchudzanie\um0427\FWLib\library\src/stm32f10x_can.c:91
   0:	2101      	movs	r1, #1
D:\STM32\Program\1.11_Odchudzanie\um0427\FWLib\library\src/stm32f10x_can.c:89
   2:	b510      	push	{r4, lr}
D:\STM32\Program\1.11_Odchudzanie\um0427\FWLib\library\src/stm32f10x_can.c:91
   4:	f04f 7000 	mov.w	r0, #33554432	; 0x2000000
   8:	f7ff fffe 	bl	0 <RCC_APB1PeriphResetCmd>
D:\STM32\Program\1.11_Odchudzanie\um0427\FWLib\library\src/stm32f10x_can.c:93
   c:	f04f 7000 	mov.w	r0, #33554432	; 0x2000000
  10:	2100      	movs	r1, #0
  12:	f7ff fffe 	bl	0 <RCC_APB1PeriphResetCmd>
D:\STM32\Program\1.11_Odchudzanie\um0427\FWLib\library\src/stm32f10x_can.c:94
  16:	bd10      	pop	{r4, pc}
